:10000000FEEF03F00000000000EF00F00000000031
:0A0010000000000000000000F3D71C
:10001C001D0E0C6E910E0D6E0D2EFED70C2EFCD7F8
:02002C001200C0
:0C002E00420E0D6E0D2EFED700001200D9
:0A003A0000000000000000001200AA
:100044004ABE02D08A9001D08A804ABC02D08A92E9
:1000540001D08A824ABA02D08A9401D08A844AB8EA
:1000640002D08A9601D08A8617B002D08A8A01D03B
:100074008A9A8A88E0DF8A984AB602D08A9001D0A8
:100084008A804AB402D08A9201D08A824AB202D0CB
:100094008A9401D08A844AB002D08A9601D08A8692
:1000A40017B002D08A8A01D08A9A8A88C4DF8A98D3
:0C00B40017A002D0B1DF01D0B8DF1200AD
:0C00C000179049C04AF0BEDF1780120004
:1000CC004450010A03E1800E446E14D04450020ADD
:1000DC0003E1C00E446E0ED04450030A03E1940EAB
:1000EC00446E08D04450040A03E1D40E446E02D08E
:1000FC00800E446E4504006E4450002600C044F04F
:10010C0000C04AF099DF1790486A48504624E96EBF
:10011C00000E4720EA6EEE50000A0BE048504624D1
:10012C00E96E000E4720EA6EEECF49F0C3DF482A95
:06013C00ECD71780120051
:100142004450010A03E1800E446E14D04450020A66
:1001520003E1C00E446E0ED04450030A03E1940E34
:10016200446E08D04450040A03E1D40E446E02D017
:10017200800E446E4504006E4450002600C044F0D8
:10018200178000C04AF05DDF179046C04AF059DF81
:0401920017801200C0
:100196008B9C8B8E010E446E010E456E2A0E2F6EC1
:1001A600200E306E410E316E4C0E326E410E336EA5
:1001B600520E346E4D0E356E450E366E200E376E6F
:1001C600490E386E4E0E396E540E3A6E520E3B6E16
:1001D600550E3C6E530E3D6E490E3E6E4F0E3F6EF3
:1001E6004E0E406E200E416E2A0E426E436A2F0E50
:1001F600466E000E476E67DF020E446E010E456EB8
:10020600200E2F6E200E306E200E316E200E326EB6
:10021600200E336E200E346E200E356E200E366E96
:10022600200E376E200E386E200E396E200E3A6E76
:10023600200E3B6E200E3C6E200E3D6E200E3E6E56
:10024600200E3F6E200E406E200E416E200E426E36
:10025600436A2F0E466E000E476E35DF030E446E60
:10026600010E456E200E2F6E200E306E200E316E62
:100276005A0E326E4F0E336E4E0E346E450E356E7E
:10028600200E366E470E376E450E386E4E0E396EA0
:10029600450E3A6E520E3B6E410E3C6E4C0E3D6E56
:1002A600450E3E6E200E3F6E200E406E200E416EB5
:1002B600200E426E436A2F0E466E000E476E03DF17
:1002C600040E446E010E456E200E2F6E200E306E0B
:1002D600200E316E200E326E200E336E200E346EDE
:1002E600200E356E200E366E200E376E200E386EBE
:1002F600200E396E200E3A6E200E3B6E200E3C6E9E
:10030600200E3D6E200E3E6E200E3F6E200E406E7D
:10031600200E416E200E426E436A2F0E466E000E70
:06032600476ED1DE12005B
:10032C0080A821D0156A80A601D019D08280828243
:10033C008284050E155CD8B08294150E0B6E4B0E94
:10034C000C6EBE0E0D6E0D2EFED70C2EFCD70B2E8A
:10035C00FAD700001550780A02E0152AE4D78290EB
:10036C00829282941ED0828082828294290E0B6E9D
:10037C00960E0C6E7F0E0D6E0D2EFED70C2EFCD72E
:10038C000B2EFAD78290A30E0B6E570E0C6E020E2C
:10039C000D6E0D2EFED70C2EFCD70B2EFAD70000AF
:0403AC008292120027
:1003B000480E4A6E47DE316A5E0E3124F66E100E2C
:1003C000F76E000EF722000EF86E000EF8220900FC
:1003D000F5CF49F075DE3150070A02E0312AECD73B
:1003E000020E4A6E2FDE2FC044F030C045F0010EE1
:0603F000466EA7DE1200BC
:1003F6009398939A93969394939293908A988A9AC1
:100406008A908A928A948A9606DE05DE04DE8A84BB
:100416008A868A880FDE8A98FEDD8A880BDE8A98AD
:10042600FADD8A8807DE8A98F6DD8A968A8802DEF1
:100436008A98F1DD8A88FEDD8A988A948A808A887D
:10044600F9DD8A98E8DD8A908A868A88F3DD8A98BB
:100456008A968A88EFDD8A98DEDD8A88EBDD8A98BF
:100466008A868A88E7DD8A98D6DD8A968A88E2DDDA
:100476008A988A808A828A848A868A88DBDD8A9834
:06048600CADD1780120020
:10048C00400E4A6ED9DD316A660E3124F66E100EBE
:10049C00F76E000EF722000EF86E000EF82209001F
:1004AC00F5CF49F007DE3150070A02E0312AECD7CC
:1004BC00020E4A6EC1DD2FC044F030C045F0466AD2
:0404CC003ADE120002
:1004D0008B8E8B9A010E446E010E456E2A0E2F6E86
:1004E000200E306E410E316E4C0E326E410E336E68
:1004F000520E346E4D0E356E450E366E200E376E32
:10050000490E386E4E0E396E540E3A6E520E3B6ED8
:10051000550E3C6E530E3D6E490E3E6E4F0E3F6EB5
:100520004E0E406E200E416E2A0E426E436A2F0E12
:10053000466E000E476ECADD020E446E010E456E19
:10054000200E2F6E200E306E200E316E200E326E79
:10055000200E336E200E346E200E356E200E366E59
:10056000200E376E200E386E200E396E200E3A6E39
:10057000200E3B6E200E3C6E200E3D6E200E3E6E19
:10058000200E3F6E200E406E200E416E200E426EF9
:10059000436A2F0E466E000E476E98DD030E446EC2
:1005A000010E456E200E2F6E200E306E5A0E316EEB
:1005B0004F0E326E4E0E336E450E346E200E356E7B
:1005C000540E366E450E376E4D0E386E500E396E27
:1005D0004F0E3A6E520E3B6E490E3C6E530E3D6E00
:1005E000450E3E6E450E3F6E200E406E200E416E53
:1005F000200E426E436A2F0E466E000E476E66DD79
:10060000040E446E010E456E200E2F6E200E306ECD
:10061000200E316E200E326E200E336E200E346EA0
:10062000200E356E200E366E200E376E200E386E80
:10063000200E396E200E3A6E200E3B6E200E3C6E60
:10064000200E3D6E200E3E6E200E3F6E200E406E40
:10065000200E416E200E426E436A2F0E466E000E33
:06066000476E34DD1200BC
:100666008B8E8B98010E446E010E456E2A0E2F6EF0
:10067600200E306E200E316E410E326E4C0E336EF1
:10068600410E346E520E356E4D0E366E450E376E79
:10069600200E386E430E396E4F0E3A6E550E3B6E77
:1006A600500E3C6E550E3D6E520E3E6E450E3F6E22
:1006B600200E406E200E416E2A0E426E436A2F0EA9
:1006C600466E000E476EFFDC020E446E010E456E4E
:1006D600200E2F6E200E306E200E316E200E326EE2
:1006E600200E336E200E346E200E356E200E366EC2
:1006F600200E376E200E386E200E396E200E3A6EA2
:10070600200E3B6E200E3C6E200E3D6E200E3E6E81
:10071600200E3F6E200E406E200E416E200E426E61
:10072600436A2F0E466E000E476ECDDC030E446EF6
:10073600010E456E200E2F6E200E306E420E316E6B
:100746004F0E326E550E336E430E346E4C0E356EB2
:10075600450E366E200E376E440E386E450E396ED7
:10076600200E3A6E470E3B6E410E3C6E520E3D6EAB
:10077600440E3E6E450E3F6E200E406E200E416EBC
:10078600200E426E436A2F0E466E000E476E9BDCAD
:10079600040E446E010E456E200E2F6E200E306E36
:1007A600200E316E200E326E200E336E200E346E09
:1007B600200E356E200E366E200E376E200E386EE9
:1007C600200E396E200E3A6E200E3B6E200E3C6EC9
:1007D600200E3D6E200E3E6E200E3F6E200E406EA9
:1007E600200E416E200E426E436A2F0E466E000E9C
:0607F600476E69DC1200F1
:1007FC000F0EC16EFF0EB46EFF0E926E946A8B8E4E
:10080C008B9C8B9A8B98829082928294EEDD010E57
:10081C004A6E12DC0C0E4A6E0FDC010E446E010E99
:10082C00456E200E1A6E430E1B6E450E1C6E4E0E40
:10083C001D6E540E1E6E520E1F6E410E206E4C0E0F
:10084C00216E450E226E200E236E200E246E440E59
:10085C00256E270E266E410E276E4C0E286E410E0D
:10086C00296E520E2A6E4D0E2B6E450E2C6E200EDE
:10087C002D6E2E6A1A0E466E000E476E21DC020E8D
:10088C00446E010E456E440E1A6E450E1B6E540ED0
:10089C001C6E450E1D6E430E1E6E540E1F6E490EC1
:1008AC00206E4F0E216E4E0E226E200E236E490EC0
:1008BC00246E4E0E256E540E266E520E276E550E5D
:1008CC00286E530E296E490E2A6E4F0E2B6E4E0E4D
:1008DC002C6E530E2D6E2E6A1A0E466E000E476E3F
:1008EC0066EC00F0030E446E010E456E200E1A6E7F
:1008FC00200E1B6E200E1C6E500E1D6E410E1E6EB9
:10090C00520E1F6E200E206E420E216E4F0E226E66
:10091C00550E236E430E246E4C0E256E450E266E20
:10092C00530E276E200E286E4E0E296E460E2A6E22
:10093C00200E2B6E200E2C6E200E2D6E2E6A1A0E93
:10094C00466E000E476E66EC00F0040E446E010E0F
:10095C00456E280E1A6E560E1B6E450E1C6E520EF0
:10096C001D6E530E1E6E490E1F6E4F0E206E4E0ED8
:10097C00216E200E226E320E236E340E246E2D0E3E
:10098C00256E300E266E390E276E2D0E286E320E09
:10099C00296E300E2A6E310E2B6E350E2C6E290EF2
:1009AC002D6E2E6A1A0E466E000E476E66EC00F027
:1009BC00186A80AA03D00A0E196E02D0140E196E92
:1009CC00660E0B6E760E0C6EC10E0D6E0D2EFED7D6
:1009DC000C2EFCD70B2EFAD78B8C8B8A8B888B9E8C
:1009EC00010E446E010E456E410E1A6E4C0E1B6EBE
:1009FC00410E1C6E520E1D6E4D0E1E6E450E1F6E60
:100A0C00200E206E480E216E4F0E226E520E236E5B
:100A1C00530E246E200E256E530E266E450E276E39
:100A2C00520E286E560E296E490E2A6E430E2B6EF0
:100A3C00450E2C6E200E2D6E2E6A1A0E466E000E72
:100A4C00476E66EC00F0020E446E010E456E440ECD
:100A5C001A6E650E1B6E6C0E1C6E610E1D6E690E91
:100A6C001E6E200E1F6E450E206E2F0E216E530E25
:100A7C00226E200E236E3A0E246E200E256E310E41
:100A8C00266E300E276E200E286E730E296E200EE9
:100A9C002A6E200E2B6E200E2C6E200E2D6E2E6AC2
:100AAC001A0E466E000E476E66EC00F0020E2F6EAC
:100ABC00020E306E77DC19500A0A67E1030E446EA1
:100ACC00010E456E200E1A6E410E1B6E540E1C6EDE
:100ADC00540E1D6E450E1E6E4E0E1F6E540E206E65
:100AEC00450E216E200E226E410E236E430E246E97
:100AFC00540E256E490E266E560E276E410E286E2C
:100B0C00540E296E490E2A6E4F0E2B6E4E0E2C6E05
:100B1C00200E2D6E2E6A1A0E466E000E476E66EC77
:100B2C0000F0040E446E010E456E200E1A6E200E5F
:100B3C001B6E200E1C6E280E1D6E470E1E6E410E77
:100B4C001F6E520E206E440E216E450E226E200E2C
:100B5C00236E410E246E430E256E540E266E490EE6
:100B6C00276E560E286E450E296E290E2A6E200E03
:100B7C002B6E200E2C6E200E2D6E2E6A1A0E466ECB
:100B8C00000E476E66EC00F09FD0020E446E010E14
:100B9C00456E440E1A6E650E1B6E6C0E1C6E610E4D
:100BAC001D6E690E1E6E200E1F6E450E206E2F0ED2
:100BBC00216E530E226E200E236E3A0E246E200EE2
:100BCC00256E320E266E300E276E200E286E730E9A
:100BDC00296E200E2A6E200E2B6E200E2C6E200EEF
:100BEC002D6E2E6A1A0E466E000E476E66EC00F0E5
:100BFC00030E446E010E456E200E1A6E410E1B6ED6
:100C0C00540E1C6E540E1D6E450E1E6E4E0E1F6E37
:100C1C00540E206E450E216E200E226E410E236E58
:100C2C00430E246E540E256E490E266E560E276EFC
:100C3C00410E286E540E296E490E2A6E4F0E2B6EE5
:100C4C004E0E2C6E200E2D6E2E6A1A0E466E000E57
:100C5C00476E66EC00F0040E446E010E456E200EDD
:100C6C001A6E200E1B6E200E1C6E280E1D6E470E6B
:100C7C001E6E410E1F6E520E206E440E216E450EDE
:100C8C00226E200E236E410E246E430E256E540EE2
:100C9C00266E490E276E560E286E450E296E290EAD
:100CAC002A6E200E2B6E200E2C6E200E2D6E2E6AB0
:100CBC001A0E466E000E476E66EC00F0020E2F6E9A
:100CCC00020E306ED8EC01F080A410D0660E0B6EC4
:100CDC00760E0C6EC10E0D6E0D2EFED70C2EFCD7A3
:100CEC000B2EFAD7BADC96EC01F0B2D180A601D06B
:100CFC0077D6010E166E1650195C2CE380A603D025
:100D0C00829082926DD680A002D0828082828B9A51
:100D1C000B0E0B6E260E0C6E5D0E0D6E0D2EFED791
:100D2C000C2EFCD70B2EFAD7000000008B8A0B0E72
:100D3C000B6E260E0C6E5D0E0D6E0D2EFED70C2E50
:100D4C00FCD70B2EFAD7000000001650191802E041
:100D5C00162AD1D780B603D080B201D005D068EC6A
:100D6C0002F096EC01F074D1070E0B6E170E0C6EA0
:100D7C006A0E0D6E0D2EFED70C2EFCD70B2EFAD74D
:100D8C000000010E446E010E456E200E1A6E200EF0
:100D9C001B6E410E1C6E4C0E1D6E410E1E6E520EC5
:100DAC001F6E4D0E206E450E216E200E226E450ECE
:100DBC00236E4E0E246E200E256E560E266E450E9C
:100DCC00276E490E286E4C0E296E4C0E2A6E450E5F
:100DDC002B6E200E2C6E200E2D6E2E6A1A0E466E69
:100DEC00000E476E66EC00F0020E446E010E456E6E
:100DFC00530E1A6E550E1B6E520E1C6E560E1D6E39
:100E0C00450E1E6E490E1F6E4C0E206E4C0E216E42
:100E1C00410E226E4E0E236E430E246E450E256E31
:100E2C00200E266E420E276E4F0E286E550E296E22
:100E3C00430E2A6E4C0E2B6E450E2C6E530E2D6EE1
:100E4C002E6A1A0E466E000E476E66EC00F01950B4
:100E5C000A0A3AE1030E446E010E456E440E1A6EF8
:100E6C00650E1B6E6C0E1C6E610E1D6E690E1E6E79
:100E7C00200E1F6E450E206E2F0E216E530E226E0D
:100E8C00200E236E3A0E246E200E256E310E266E29
:100E9C00300E276E200E286E730E296E200E2A6ED1
:100EAC00200E2B6E200E2C6E200E2D6E2E6A1A0E1E
:100EBC00466E000E476E66EC00F0030E2F6E020EAF
:100ECC00306ED8EC01F039D0030E446E010E456E35
:100EDC00440E1A6E650E1B6E6C0E1C6E610E1D6E32
:100EEC00690E1E6E200E1F6E450E206E2F0E216E8B
:100EFC00530E226E200E236E3A0E246E200E256E9B
:100F0C00320E266E300E276E200E286E730E296E52
:100F1C00200E2A6E200E2B6E200E2C6E200E2D6EA7
:100F2C002E6A1A0E466E000E476E66EC00F0030E2B
:100F3C002F6E020E306ED8EC01F0040E446E010ED2
:100F4C00456E200E1A6E200E1B6E200E1C6E200E8F
:100F5C001D6E200E1E6E200E1F6E200E206E200E9B
:100F6C00216E200E226E200E236E200E246E200E7B
:100F7C00256E200E266E200E276E200E286E200E5B
:100F8C00296E200E2A6E200E2B6E200E2C6E200E3B
:100F9C002D6E2E6A1A0E466E000E476E66EC00F031
:100FAC00182A040E2F6E18C030F046EC02F01850C0
:100FBC00140AD8B4186A80A230D0010E166E1650DE
:100FCC00195C26E38B9A0B0E0B6E260E0C6E5D0EC7
:100FDC000D6E0D2EFED70C2EFCD70B2EFAD7000063
:100FEC0000008B8A0B0E0B6E260E0C6E5D0E0D6EBA
:100FFC000D2EFED70C2EFCD70B2EFAD700000000BE
:10100C0080A601D0EDD41650191802E0162AD7D7B5
:10101C0068EC02F096EC01F01BD080A411D0660EA7
:10102C000B6E760E0C6EC10E0D6E0D2EFED70C2EA9
:10103C00FCD70B2EFAD733EC03F096EC01F008D06A
:10104C0080A005D0CBEC00F096EC01F001D08CD652
:02105C00FFD7BC
:08105E0002040E111F100E0028
:08106600181C1E1F1F1E1C18A0
:020000040030CA
:0D000100021F1EFF8381FF0FC00FE00F40A4
:00000001FF
